:100000000C9438000C9466000C94ED000C94530092
:100010000C9453000C9453000C9453000C94530014
:100020000C9453000C9453000C9453000C94530004
:100030000C9453000C9453000C9453000C945500F2
:100040000C9453000C9453000C9453000C945300E4
:100050000C9453000C9453000C9453000C945300D4
:100060000C9453000C9453000C9453000C945300C4
:1000700011241FBECFEFD0E1DEBFCDBF12E0A0E064
:10008000B1E0EEE9FDE002C005900D92A638B1079F
:10009000D9F71EE0A6E8B2E001C01D92A23FB10769
:1000A000E1F70C9442030C9400001F920F920FB6DC
:1000B0000F9211248F93809186028F5F8093860226
:1000C0008F910F900FBE0F901F9018951F920F9257
:1000D0000FB60F9211248F939F93EF93FF93E091AC
:1000E0008702FF278091840090918500EE0FFF1F0B
:1000F000EE56FD4F91838083E0918702FF27809128
:100100008602EE53FD4F8083E0918702FF27E6527F
:10011000F14F81E08083E0918702FF2780911001F9
:10012000F695FE2FEE27F795E795E652FD4F808B6B
:10013000E0918702FF2780911101F695FE2FEE27AF
:10014000F795E795E652FD4F818BE0918702FF27F7
:1001500080911201F695FE2FEE27F795E795E6526E
:10016000FD4F828BE0918702FF2780911301F69566
:10017000FE2FEE27F795E795E652FD4F838BE09132
:100180008702FF2780911401F695FE2FEE27F79541
:10019000E795E652FD4F848BE0918702FF2780911F
:1001A0001501F695FE2FEE27F795E795E652FD4FE0
:1001B000858B809187028F5F809387028091870271
:1001C000883111F410928702FF91EF919F918F91E6
:1001D0000F900FBE0F901F9018951F920F920FB6A1
:1001E0000F9211242F933F934F935F936F937F93BD
:1001F0008F939F93EF93FF931DBA87E788B988B9D0
:100200008FEF88B986B18171E9F3E0918702FF270A
:100210008091840090918500EE0FFF1FEE56FD4FF8
:1002200091838083E0918702FF2780918602EE53BD
:10023000FD4F808386B18171E9F789E988B988B972
:1002400088B988B990B153B18FEF88B921E030E017
:1002500077E76FEF49E978B978B968B986B1817104
:10026000E9F3E0918702FF27F695FE2FEE27F79539
:10027000E795E20FF31FE752FD4F9083E09187026D
:10028000FF27F695FE2FEE27F795E795E652FD4FEF
:10029000E20FF31F508386B18171E9F748B948B97D
:1002A00048B948B990B153B168B92E5F3F4F2F3765
:1002B000310589F6E0918702FF27F695FE2FEE279C
:1002C000F795E795E85AFC4F9083E0918702FF2766
:1002D000F695FE2FEE27F795E795E75AFC4F5083EA
:1002E000E0918702FF27E652F14F32E03083209100
:1002F0008702809187028F5F8093870280918702B7
:100300008831B9F090918702809188029817C9F0DE
:10031000809189028F5F8093890280918902803168
:1003200020F43CBB83E08DBB0FC03CBB81E08DBBA8
:100330000BC01092870290918702809188029817D3
:1003400039F720938702E4CFFF91EF919F918F912E
:100350007F916F915F914F913F912F910F900FBEC1
:100360000F901F9018958F708A3018F0895C99272C
:100370000895805D9927089560E070E0809185027E
:100380008F7E8093850220E030E040E050E0809155
:1003900085028BB92F5F3F4F4F4F5F4F203888E367
:1003A000380781E0480780E0580789F78091850287
:1003B00080618093850220E030E040E050E0809151
:1003C00085028BB92F5F3F4F4F4F5F4F203888E337
:1003D000380781E0480780E0580789F78091850257
:1003E0008F7D8093850220E030E040E050E08091F6
:1003F00085028BB92F5F3F4F4F4F5F4F203888E307
:10040000380781E0480780E0580789F78091850226
:1004100080628093850220E030E040E050E08091EF
:1004200085028BB92F5F3F4F4F4F5F4F203888E3D6
:10043000380781E0480780E0580789F780918502F6
:100440008F7B8093850220E030E040E050E0809197
:1004500085028BB92F5F3F4F4F4F5F4F203888E3A6
:10046000380781E0480780E0580789F780918502C6
:1004700080648093850220E030E040E050E080918D
:1004800085028BB92F5F3F4F4F4F5F4F203888E376
:10049000380781E0480780E0580789F76F5F7F4F92
:1004A0006430710509F06ACF0895982F80918B020E
:1004B000873028F5292F332780918B02E09179022C
:1004C000F0917A02E80FF11D8081992787FD9095C0
:1004D0002817390709F446C041E080918B02E0916A
:1004E0008302F0918402E80FF11D8081992787FD36
:1004F00090952817390709F44BC0442341F58091A2
:100500008B028F5F80938B0280918B02873080F00B
:1005100010928B0280918F02873058F48091900264
:10052000873038F5109290028091900280938F026C
:100530000895109290028091900280938F02809192
:100540008A028F5F80938A0210928E020895109221
:100550008B0280918B028093900280919002809315
:100560008F02089580918F028F5F80938F0240E009
:10057000B4CF109290028091900280938F0280916C
:100580008A028F5F80938A0281E080938E020895B1
:10059000809190028F5F80939002B1CF982F8C3220
:1005A000A1F080918B02841778F480918B02262F22
:1005B000280F312D311DF901E050FF4F90838091BC
:1005C0008B028F5F80938B02089580918A028F5FE8
:1005D00080938A0210928B020895982F8C32C9F072
:1005E00080918B028417A0F480918B02262F280F14
:1005F000312D311DF901E050FF4F908380918B0226
:100600008F5F80938B029E3219F481E08093910278
:10061000089580918A028F5F80938A0280918B0275
:10062000841758F580919102882381F480918B0280
:10063000262F280F312D311DF901E050FF4F8EE29A
:10064000808380918B028F5F80938B0280918B02DD
:10065000841798F4772790E380918B02FB01E80FD1
:10066000F11DE050FF4F908380918B028F5F80934C
:100670008B0280918B02841778F310929102109272
:100680008B020895CFEFD0E1DEBFCDBF11B89FEF51
:1006900092B914B895B98EE087B998B980E78AB94C
:1006A0008FE88BB982E08093810081E080936F00B6
:1006B00015BE8BE08093690083E08DBB789416B102
:1006C000107C0E94BC01103409F466C3103809F490
:1006D00060C3112309F05AC390E08FE19093C500E5
:1006E0008093C40088E18093C10086E08093C200BB
:1006F000A0916F02B09170028C91882369F0FD0186
:1007000031968091C00085FFFCCF8C918093C6000C
:10071000DF0181918823A9F7FF248091C00087FD24
:1007200056C090918702809188029817B1F3E091AA
:100730008802FF27E652F14F8081813009F467C0BB
:10074000E0918802FF27E652F14F8081823029F73D
:1007500080918C0290918D02892B09F4C0C1809107
:100760008C0290918D02019709F438C280918C021D
:1007700090918D02029708F46FC180918C02909144
:100780008D028151914008F067C18091C00085FFC2
:10079000C4CFE0918C02F0918D02EC5BFE4F808122
:1007A0008093C600E0918C02F0918D02EC5BFE4FCD
:1007B0008081F82680918C0290918D020196909311
:1007C0008D0280938C028091C00087FFAACF909108
:1007D000C60080918A02882309F4D0C080918E02DD
:1007E000882309F0B6C080918A02853009F448C296
:1007F000863008F022C2823009F491C2833008F0BA
:1008000070C2813009F4B0C210928A028ACF8091FE
:100810008C0290918D02892B09F4B4C080918C02D6
:1008200090918D02892BD1F080918C0290918D0254
:100830004197A0F48091C00085FF6FCFE0918C02BA
:10084000F0918D02E150FF4F80818093C600E091CE
:100850008C02F0918D02E150FF4FAACF80918C0263
:1008600090918D02419770F180918C0290918D0250
:10087000479740F58091C00085FF4FCF8091880257
:100880009927E0918C02F0918D029695982F8827F8
:1008900097958795E80FF91FE752FD4F8081809368
:1008A000C600809188029927E0918C02F0918D0218
:1008B0009695982F882797958795E80FF91FE75207
:1008C000FD4F76CF80918C0290918D02479740F03A
:1008D00080918C0290918D028634910508F4AACF04
:1008E00080918C0290918D028634910509F461C14A
:1008F00080918C0290918D028734910509F4C6C1D4
:1009000080918C0290918D028834910509F4C4C1C4
:1009100080918C0290918D028934910509F4CDC1AA
:1009200080918502806480938502809185028BB9D5
:1009300010928D0210928C02809188028F5F8093BA
:10094000880280918802883109F408C283E08DBB57
:10095000E4CE80918A02853059F0863008F07FC15C
:10096000823031F0833008F0CEC1813009F04CCFB5
:1009700040E060E0892F0E94CE02D3CE892F0E94F2
:100980005502CFCE809185028F7B80938502809126
:1009900085028BB9E0918802FF27EE53FD4F8081DD
:1009A00082958F700E94B30180930701E0918802C5
:1009B000FF27EE53FD4F80810E94B3018093080111
:1009C000E0918802FF27EE0FFF1FEE56FD4F80815A
:1009D0009181892F992782958F700E94B30180930E
:1009E0000901E0918802FF27EE0FFF1FEE56FD4F31
:1009F00080819181892F99270E94B30180930A01F8
:100A0000E0918802FF27EE0FFF1FEE56FD4F808119
:100A10009181929582958F7089279F7089270E9476
:100A2000B30180930B01E0918802FF27EE0FFF1FB7
:100A3000EE56FD4F808191810E94B30180930C019D
:100A400080918C0290918D02019690938D028093FB
:100A50008C020EE0F02E61CE80918C0290918D027E
:100A60008151914009F4A5C080918C0290918D0232
:100A70008251914009F40AC180918C0290918D02BB
:100A80008351914009F408C180918C0290918D02AC
:100A90008451914009F411C1809185028061809355
:100AA0008502809185028BB910928D0210928C0282
:100AB000809188028F5F80938802809188028831BC
:100AC00009F44FC1809189028150809389028091FD
:100AD0008902803108F021CE82E08CBB37CF809133
:100AE00085028F7E80938502809185028BB9E0918B
:100AF0008802FF27EE53FD4F808182958F700E9400
:100B0000B30180934D01E0918802FF27EE53FD4F22
:100B100080810E94B30180934E01E0918802FF27FB
:100B2000EE0FFF1FEE56FD4F80819181892F99278F
:100B300082958F700E94B30180934F01E0918802EB
:100B4000FF27EE0FFF1FEE56FD4F80819181892F09
:100B500099270E94B30180935001E0918802FF27FA
:100B6000EE0FFF1FEE56FD4F808191819295829589
:100B70008F7089279F7089270E94B301809351014C
:100B8000E0918802FF27EE0FFF1FEE56FD4F808198
:100B900091810E94B3018093520180918C029091C7
:100BA0008D02019690938D0280938C022EE0F22E9E
:100BB000B4CD8091C00085FFB0CD8F2D82958F7010
:100BC0000E94B3018093C60080918C0290918D02A7
:100BD000019690938D0280938C029FCDC0E0D0E06F
:100BE00004E511E0E0918802FF27F695FE2FEE273D
:100BF000F795E795E652FD4FEC0FFD1F808182953A
:100C00008F700E94B301F8018083E0918802FF2772
:100C1000F695FE2FEE27F795E795E652FD4FEC0F80
:100C2000FD1F808121960E94B301F80181830E5F30
:100C30001F4FC038D105B1F6BDCD873009F498CE2D
:100C4000873008F45AC0883009F492CE893009F010
:100C5000DBCD46E067E1892F0E94CE0262CD88306D
:100C600009F486CE893088F5863009F481CE873044
:100C700009F0CACD42E062E4892F0E94CE0251CD34
:100C80004AE06AE2892F0E94CE024BCD8091C000DB
:100C900085FF43CD8F2D94CF8091C00085FF3DCD42
:100CA0008DE08093C60080918C0290918D02019618
:100CB00090938D0280938C0230CD8091C00085FF8F
:100CC0002CCD8AE08093C60075CD893009F458C0D8
:100CD0008A3009F099CD41E060E4892F0E94CE026C
:100CE00020CD833009F446C0843009F08DCD41E039
:100CF00068E2892F0E94CE0214CD41E065E3892F7E
:100D00000E94CE020ECD833009F432CE843009F039
:100D10007BCD40E060E0892F0E94CE0202CD41E011
:100D20006EE0892F0E94CE0280910E01813469F01D
:100D30008091150180FD09C08091850280628093B9
:100D40008502809185028BB9ECCC809185028F7DE4
:100D500080938502809185028BB9E3CC1092880242
:100D6000F5CD10928802AECE46E060E1892F0E9458
:100D7000CE02D7CC49E06EE1892F0E94CE02D1CCC1
:100D800048E067E3892F0E94ED02CBCC91E083E03D
:0E0D9000A5CC90E080E4A2CC90E081E89FCC5E
:100D9E0024424C5345432C3030303030302C2D2CE7
:100DAE003030303030302C3030303030302C30303D
:100DBE0030302E303030302C4E2C30303030302E13
:100DCE00303030302C452C30303030303030302C0C
:100DDE004D2C30302A0024424C5345512C303030AB
:100DEE003030302C303030303030303030303030F9
:100DFE0030303030303030303030303030303030E5
:100E0E0030303030303030303030303030303030D4
:100E1E0030303030303030303030303030303030C4
:100E2E0030303030303030303030303030303030B4
:100E3E0030303030303030303030303030303030A4
:100E4E003030303030303030303030303030303094
:100E5E003030303030303030303030303030303084
:100E6E003030303030303030303030303030303074
:100E7E003030303030303030303030303030303064
:100E8E003030303030303030303030303030303054
:100E9E003030303030303030303030303030303044
:100EAE003030303030303030303030303030303034
:100EBE003030303030303030303030303030303024
:100ECE003030303030303030303030303030303014
:100EDE003030303030303030303030303030303004
:100EEE00303030302A000D0A4669726D77617265B6
:100EFE002056657273696F6E3A2032350D0A0056B0
:100F0E0002244750524D432C00710224475047474C
:060F1E00412C007B02FFE4
:00000001FF
